:040000008A15D62F58
:08000800FF00030E8312031335
:10001000E8000A0EE900040EEA008A110A16032815
:100020000330AF07AF0CAF0C7F30AF050000AF0B54
:1000300016280800A108031D1E280800F930FF3EFD
:10004000031D1F280000A10B1E280800000000004F
:1000500000000000000000000000A40B262808009B
:10006000D008031D3628D10803190800203050029B
:10007000510803185428031D542845125008D20073
:100080008312501C45288316451603108312D30C87
:10009000D20CD10CD00C8316D203031D4028451E70
:1000A00008008312501408008312500851045204AF
:1000B0005304FF39031908000130D000D101D201E7
:1000C000D301080083160313D2014030D300F00897
:1000D000031D6C280130D200D208031D822870084D
:1000E000033A031D7528D30182287F30D300F60818
:1000F00003197F287008023A0319D301822870037C
:100100000319D301831254088316D60083125508AD
:100110008316D700831256088316D8008312570817
:100120008316D9005308DA00DB01DC01DD01D31F9F
:100130009C28DB03DC03DD035A08D6075B080318A1
:100140005B0FD7075C0803185C0FD8075D0803181E
:100150005D0FD9077F30831254058316D400003019
:1001600083126C02031DB628FD306B02031C632949
:100170006B08FD3C6C080318031DEC1BC028C92844
:10018000FD306B0603196C08031DE3288316D91F85
:10019000E3282830F1048316D308031DDA287F30C2
:1001A0008312D600FF30D400D500D701FE30EB001B
:1001B000EC010800FF308312EB00EC01D401D50103
:1001C000D601D70108008312EC1F63298316DB01D7
:1001D00083126F03031DEE288316DB0A8316DA01F0
:1001E00083126C08803A8316DF007F305F02031DA4
:1001F000FC28FF3083126B02031800298316DA0AE9
:100200008316DE01DA080319DB08031DDE0A8030DD
:100210005905DC00DD01DD0ADC08031D5D10D50198
:10022000DD080319DE08031DD50A8312EB08031944
:10023000EC08031955296B098316DA0083126C093F
:100240008316DB00DA0A0319DB0A20305A025B0846
:1002500003182C2903192E29DB1F48295C1083124F
:100260006B098316DD00DD0A8312541C39298316BD
:100270005C1403108312D70CD60CD50CD40C831647
:10028000DD03031D34295C1C5529831254145529A0
:1002900083125408550456045704FF39031955298D
:1002A0000130D400D501D601D7018312EB01EC0156
:1002B0007F3054058316D400D50803196329D40868
:1002C0000319632971168316D408031DF116530808
:1002D000DA00DB01DC01DD01D31F7129DB03DC0364
:1002E000DD035A088312D40783165B08031C7B299D
:1002F0005B0F7B297D298312D50783165C08031CBD
:1003000084295C0F842986298312D60783165D0809
:10031000031C8D295D0F8D298F298312D707073084
:100320008316DA00DA0803199E2903108312D70C0A
:10033000D60CD50CD40C8316DA039229403054061F
:10034000031DA729D2080319A72983125410831269
:100350005408550456045704FF39031D0800EB01E7
:10036000EC01080083120313571CBA290230EB0773
:100370000318EC0AD61FC029EB0A031DC029EC0A9A
:100380006B08D7000310D70CD6136B18D617F608D6
:10039000031DD7170800403083160313CA00D2018B
:1003A000D301D401D5018312D401D501D601D701DF
:1003B00083164A08CB00CA03CB0803193A2A031054
:1003C0008312D40DD50DD60DD70D8316D51FEA296E
:1003D0008312541403108316D20DD30DD40DD50DF2
:1003E0008312D31F312A4C088316D20783124D087B
:1003F000031CFD294D0FFD29FF298316D307831206
:100400004E08031C062A4E0F062A082A8316D40714
:1004100083124F08031C0F2A4F0F0F2A112A83162D
:10042000D50783124F0883165502031D272A83120E
:100430004E0883165402031D272A83124D08831683
:100440005302031D272A83124C08831652020318F5
:10045000312A8312D40A0319D50A0319D60A0319BB
:10046000D70A8312D71B3A2A0310D00DD10DD20D13
:10047000D30DD8298312EC01203083164A0283124F
:10048000EB00031CEC038316CA1F482A8312EC03FB
:1004900083165208530454045504FF390319080005
:1004A000831254140800831203134C08D4004D081F
:1004B000D5004E08D6004F08D700750874060319FA
:1004C000942A5008003C8316D0000030D100D2009E
:1004D000D300831251080318702A510F702A722A10
:1004E0008316D102831252080318792A520F792AEF
:1004F0007B2A8316D202831253080318822A530FD1
:10050000822A842A8316D302831650088312D000CD
:10051000831651088312D100831652088312D20029
:10052000831653088312D3005008D40751080318C8
:10053000510FD50752080318520FD6075308031856
:10054000530FD707F7015408550456045704FF39D1
:10055000031D08000130F7000800D601D701D801BB
:10056000D901DA01D61A08004E1CC42A4A08D70756
:100570004B0803184B0FD8074C0803184C0FD9072A
:100580004D0803184D0FDA070310D10CD00CCF0C17
:10059000CE0C0310CA0DCB0DCC0DCD0DD60AB22A50
:1005A000D201D301D401D501D701D801D901DA0193
:1005B000D601D61A08000310D70DD80DD90DDA0DC3
:1005C000CA0DCB0DCC0DCD0DD20DD30DD40DD50D47
:1005D00051085502031DF62A50085402031DF62A3D
:1005E0004F085302031DF62A4E085202031C072B24
:1005F0004E08D2024F08031C4F0FD3025008031CB1
:10060000500FD4025108031C510FD5025714D60ABB
:10061000D92A831203135408550456045704FF398A
:1006200003191E2B571B08000310D40DD50DD60D32
:10063000D70DEB080319EC03EB03122BEB01EC01D4
:1006400008003C088312CC0083163D088312CD00BD
:1006500083163E088312CE00CE13CF0183163F08C7
:10066000F200F2130310F20DBE1B7214F401BF1F4F
:100670003B2B0130F400C10196307202C000031C14
:10068000C10380307202C2004208153C0318DC2B03
:10069000C21BDC2B42081D3C0318812BC21B812B83
:1006A0003C08003C031D602B3D08003C031D602BF3
:1006B0003E08003C031D602B3F08CF3C03197A2BFA
:1006C0007114F4080319722B42087F3AC21B7A2B6B
:1006D000031D7A2B83124C084D044E044F04FF393E
:1006E00003197A2B7F308316CA00FF30C700C80079
:1006F000C90008008316C701C801C9018030CA00BB
:1007000008001630C2028312CE1783164208CB00AF
:10071000CB080319942B03108312CC0DCD0DCE0DF5
:10072000CF0D8316CB03882BF4080319CB2B831230
:100730004C08003C8316CB000030CC00CD00CE002E
:1007400083124D080318A72B4D0FA72BA92B831637
:10075000CC0283124E080318B02B4E0FB02BB22BD5
:100760008316CD0283124F080318B92B4F0FB92BF4
:10077000BB2B8316CE0283164B088312CC00831644
:100780004C088312CD0083164D088312CE008316C9
:100790004E088312CF0083124C088316C7008312C1
:1007A0004D088316C80083124E088316C9008312B1
:1007B0004F088316CA0008007E3072020318FD2B12
:1007C000F2080319E42BEC2B83124C084D044E0461
:1007D0004F04FF390319F32B01308316CB00CC01F2
:1007E000CD01CE01F82B8316CB01CC01CD01CE017A
:1007F000C301C401C501C6013C2C8312CE174C08AD
:100800008316CB0083124D088316CC0083124E084A
:100810008316CD0083124F088316CE001F3040058B
:10082000CF00CF0803191B2C0310CB0DCC0DCD0D21
:10083000CE0DCF03112C83124C088316C3008312F4
:100840004D088316C40083124E088316C500831218
:100850004F088316C600C009C109C00A0319C10A9E
:100860004008CF00CF0803193C2C460DC60CC50C20
:10087000C40CC30CCF03322C4B084C044D044E0463
:10088000FF39031DF116F008031D842CCE1F652CC3
:10089000C30A0319C40A0319C50A0319C60A4B0877
:1008A000CF004C08D0004D08D1004E08D2000310F4
:1008B000CF0DD00DD10DD20D4F085004510452046C
:1008C000FF39031D652CFE30C305F4080319C62C3F
:1008D0004308003CCF000030D000D100D2004408D3
:1008E000031C440FD0024508031C450FD1024608E3
:1008F000031C460FD2024F08C3005008C400510821
:10090000C5005208C600C62CCF014B084C044D044C
:100910004E04FF39031D4F14F4080319B82C70035B
:10092000031D9C2CCF0803199C2CC30A0319C40A6D
:100930000319C50A0319C60A4308003CD000003059
:10094000D100D200D3004408031C440FD102450853
:10095000031C450FD2024608031C460FD302500861
:10096000C3005108C4005208C5005308C600C62C75
:100970007008023A031DC62CCF080319C62CC30AFF
:100980000319C40A0319C50A0319C60A4308C70094
:100990004408C8004508C9004608CA0008003C08C9
:1009A0008312CC0083163D088312CD0083163E08C7
:1009B0008312CE00CE13CF0183163F08F200F2134C
:1009C0000310F20DBE1B721440088312D000831670
:1009D00041088312D100831642088312D200D21339
:1009E000D30183164308F300F3130310F30DC21B66
:1009F0007314F401BF1FFE2C0130F400F501C31F76
:100A0000032D0130F50075087406F6004410720AD3
:100A100003194414C410730A0319C4144411831233
:100A20004C084D044E044F04FF39031D192D831645
:100A300044158316C4118312500851045204530400
:100A4000FF39031D252D8316C415831644182A2D3E
:100A5000C41C712D441C322D4419322D3E1B322DE5
:100A60007114622DC41C3A2DC4193A2D421B3A2D23
:100A70007114622D441C3E2D441D622DC41C422D58
:100A8000C41D622DC41D492DF308031D492D711489
:100A9000622D441D502DF208031D502D7114622D3E
:100AA000CA01CB017F30CD008030CC00F608031D99
:100AB000CD174D08D1004C08D0004B08CF004A0894
:100AC000CE000800CA01CB01C030CC00FF30CD0001
:100AD0004D08D1004C08D0004B08CF004A08CE008A
:100AE00008007F30C500F208031D942D441D882D99
:100AF000CA01CB01CD01CC01F608031DCD174D086D
:100B0000D1004C08D0004B08CF004A08CE000800A6
:100B1000C5038312CE1B962D0310CC0DCD0DCE0D2B
:100B2000CF0D8316C50A892D8312CE17F308031D36
:100B3000B82D8316C41DAC2DCA01CB01CD01CC014B
:100B4000F608031DCD174D08D1004C08D0004B0806
:100B5000CF004A08CE000800C5038312D21BB92D6E
:100B60000310D00DD10DD20DD30D8316C50AAD2DB6
:100B7000D21707308316CA00CA080319C82D0310FC
:100B80008312CC0DCD0DCE0DCF0D8316CA03BC2D17
:100B90000830CA00CA080319D62D03108312D00DDD
:100BA000D10DD20DD30D8316CA03CA2DCB218312CA
:100BB000EB080319EC080319172E6B098316CA00FA
:100BC00083126C098316CB00CA0A0319CB0A2030A2
:100BD0004A024B080318EE2D0319F02DCB1F0A2EE5
:100BE000441283126B098316CC00CC0A8312541C66
:100BF000FB2D8316441603108312D70CD60CD50C8C
:100C0000D40C8316CC03031DF62D441E172E83121D
:100C10005414172E83125408550456045704FF39F0
:100C20000319172E0130D400D501D601D70172085F
:100C30008312EB00EC017308EB070318EC0A831630
:100C400045088312EB02031CEC03571B302E0310E4
:100C5000D40DD50DD60DD70DEB080319EC03EB031E
:100C60006220B22154088316C600831255088316E9
:100C7000C700831256088316C800831257088316CC
:100C8000C9004908D1004808D0004708CF004608ED
:100C9000CE0008003F08DD003E08DC003D08DB0018
:100CA0003C08DA005D08DE000310DE0DDC1B5E147C
:100CB0005E08C600C701FF30460603194708031D3A
:100CC0007A2E3F08DD003E08DC003D08DB003C08D2
:100CD000DA00DC13DD015A08C8005B08C9005C08B3
:100CE000CA005D08CB00480849044A044B04FF3998
:100CF000031DAA2E4308DD004208DC004108DB008A
:100D00004008DA005D08DE000310DE0DDC1B5E1417
:100D10005E08CC00CD01FF304C0603194D08031DC1
:100D2000AD2E4308DD004208DC004108DB0040082E
:100D3000DA00DC13DD015A08CE005B08CF005C0846
:100D4000D0005D08D1004E084F0450045104FF3913
:100D50000319AD2E7114DA0108003F08DE003E08C9
:100D6000DD003D08DC003C08DB0080305E05DF0074
:100D7000C401DF08031D44144308DE004208DD00FF
:100D80004108DC004008DB0080305E05DF00C50163
:100D9000DF08031D4514450844060319F72E4008D3
:100DA0003C04D20041083D04D30042083E04D40074
:100DB00043083F04D5000310D20DD30DD40DD50D3B
:100DC000D601D60AD208031D5610D308031D5610AB
:100DD000D408031D5610D508031D5610DB01D60894
:100DE0000319C408031DDB0A5B08DA000800D901F7
:100DF000D90A40083C02031DD90141083D02031DE8
:100E0000D90142083E02031DD90143083F02031DD8
:100E1000D901D70143083F02031D182F42083E02A3
:100E2000031D182F41083D02031D182F40083C02E6
:100E3000031CD70A57084406D800DB01D808031959
:100E4000D908031DDB0A5B08DA0008004408831296
:100E5000D400831645088312D500831646088312F2
:100E6000D600831647088312D7005408003C031DA0
:100E70004B2F5508003C031D4B2F5608003C031D0B
:100E80004B2F5708803C031D4B2F0130F6009E303E
:100E9000EB00EC01882FF601D71F832F0130F600FD
:100EA0005408003C8316CC000030CD00CE00CF00AB
:100EB0008312550803185F2F550F5F2F612F83167C
:100EC000CD02831256080318682F560F682F6A2F19
:100ED0008316CE02831257080318712F570F712FF4
:100EE000732F8316CF0283164C088312D400831607
:100EF0004D088312D50083164E088312D600831640
:100F00004F088312D7009C30EB00EC0109236220CC
:100F1000B22154088316C800831255088316C900ED
:100F2000831256088316CA00831257088316CB0013
:100F30004B08CF004A08CE004908CD004808CC0035
:100F40000800C4080319A62F8030C3063F08F2002A
:100F5000F2130310F20DBE1B7214F401BF1FB22F67
:100F60000130F4003C088312CC0083163D08831244
:100F7000CD0083163E088312CE00CE13CF01831618
:100F80004308F300F3130310F30DC21B7314F501B0
:100F9000C31FCC2F0130F50040088312D000831608
:100FA00041088312D100831642088312D200D21363
:100FB000D30106308316CC00CC080319E82F0310A8
:100FC0008312CC0DCD0DCE0DCF0D8316CC03DC2FAF
:100FD0000630CC00CC080319F62F03108312D00D75
:100FE000D10DD20DD30D8316CC03EA2F4510720A12
:100FF00003194514C510730A0319C514451183124A
:101000004C084D044E044F04FF398A15031D0A286D
:10101000831645158316C5118312500851045204D6
:101020005304FF39031D16288316C515831645186A
:101030001B28C51C76284516421F1F284512C516B9
:101040003E1BC512451C4228C51C4228451D33289D
:10105000C51D332875087406031963287114F40834
:10106000031D62286C28451D3A28C5193A28451ADF
:1010700071146C2845194228C51D4228C51E6228D6
:1010800071146228451C4828451D4828C51C632842
:10109000C51C4E28C51D4E28451C6D28451C5B28C7
:1010A00045195B28C51A7114C51C6228C519622828
:1010B000451A71146228C51C6228C5196228451A90
:1010C00071146C283E173F08CF003E08CE003D0843
:1010D000CD003C08CC00080042174308CF0042086E
:1010E000CE004108CD004008CC0008007208C600C0
:1010F000C7017308D000D1015008C602510A031875
:101100005108C70273087202031C9B2872087306F9
:10111000031DC728831253084F02031D9928520844
:101120004E02031D992851084D02031D99285008AD
:101130004C020318C72883124F08D7004E08D60068
:101140004D08D5004C08D4007208EB00EC0174087F
:10115000F6005308CF005208CE005108CD005008C9
:10116000CC005708D3005608D2005508D1005408C7
:10117000D0007308F2006B08F3007508F4007608DD
:10118000F5008316C609C709C60A0319C70AF2087B
:10119000031DF428F308031DF4288A115322F708CD
:1011A0008A150319DF28750874060319DF287003F0
:1011B000031DDD280130F600E128F601E12874085E
:1011C000F60006308316D000D0080319F02803106B
:1011D0008312D70CD60CD50CD40C8316D003E4287C
:1011E0008312EB01EC013229F308031DFE2883165C
:1011F000C608031DFC28C703C60300298312D316A3
:10120000F208031D09298316C60A031D0B29C70A04
:101210000B298312CF1683164608D0004708D10049
:101220008A1130205322F7088A1503191F297003E9
:10123000031D1D290130F6002129F601212974081A
:10124000F6007208EB00EC01571B2F290310D40D98
:10125000D50DD60DD70DEB080319EC03EB038A115E
:10126000092362208A11B22154088316C800831210
:1012700055088316C900831256088316CA008312C4
:1012800057088316CB004B08CF004A08CE00490808
:10129000CD004808CC00080083160313A0017E0887
:1012A00020020318080064000130A1008A111A20EE
:1012B000A00A8A154F290430831203131F049F00CC
:1012C0001F196029FE08031978291E088316AC002F
:1012D000AD01AC0DAD0DAC0DAD0DFC30AC051E0C73
:1012E000AE00AE0CAE0E03302E05AC04AD087C296A
:1012F0001E088316AC00AD012C08AE002D08AF000F
:1013000008007E08003A03198929013A03199A292D
:10131000AE290130FB0000308312EE008530ED0075
:101320008316AD08031D97290E309F00AE290530A6
:101330009F00AE290230FB000030AF0085308312E1
:10134000ED0083162F088312EE008316AD08031DEF
:10135000AC2904309F00AE2905309F002C08033CC7
:10136000031C1F17831383126E1883176D088400E4
:101370000008FA007B087A048316AF0080002C086E
:10138000AF00B001AF0DB00DAF0DB00DAF0DB00D92
:10139000AF0DB00DAF0DB00DAF0DB00DC0302F05BE
:1013A0000138B2007E08B100B10DB10DB10DF830B9
:1013B0003105320483129F0083162E08AF008A1174
:1013C000102008008313831203136E1883176D080F
:1013D00084007A088000073083169F0083129F01E3
:1013E0000800C208031DF629C9010800C401CA305B
:1013F000C5009A30C6003B30C700C801BF1F162A7F
:1014000083134118831740088400CA014A088407DF
:101410002D308000C80ABC09BD09BE09BF09BC0F38
:10142000162ABD0F162ABE0F162ABF0AC3013C0892
:101430003D043E043F04FF39031D242A0130C3004C
:10144000C400C501C601C701420848020318AA2A00
:101450004708003C031D362A4608003C031D362A77
:101460004508003C031D362A4408003C0318AA2AFC
:1014700047083F02031D462A46083E02031D462A2E
:1014800045083D02031D462A44083C0203184B2A26
:10149000C3080319912A3C08CA003D08CB003E0846
:1014A000CC003F08CD004408CE004508CF004608D8
:1014B000D0004708D1008A11D0225708C300430842
:1014C000303ECA0083134118831740084807840040
:1014D0004A088000C80A4308CA00CB01CC01CD01EC
:1014E0004408CE004508CF004608D0004708D10088
:1014F000AD225708D2005808D3005908D4005A0822
:10150000D5005208BC025308031C530FBD025408F7
:10151000031C540FBE025508031C550FBF020130B7
:10152000C3004408CA004508CB004608CC00470861
:10153000CD000A30CE00CF01D001D1018A11D022D6
:101540005708C4005808C5005908C6005A08C70003
:101550008A15242A420848020318B62A8313411820
:101560008317400848078400003080004808C900FD
:1015700008008312861106118610061086120612C4
:101580008316210E0F39A3000F30A305231CCA2A8E
:10159000831286158316A31CCF2A83120615831681
:1015A000231DD42A831286148316A31DD92A8312DD
:1015B00006148316A2080319DF2A831286160A303E
:1015C0008316A4008A112620831206160A30831679
:1015D000A4002620831206120F3083162105A300D3
:1015E0000A30A400262083128611061186100610E8
:1015F0008612061283168A15231C002B8312861569
:101600008316A31C052B831206158316231D0A2B94
:10161000831286148316A31D0F2B831206148316C0
:10162000A2080319152B831286160A308316A4000C
:101630008A112620831206160A308316A40026205B
:10164000831206120A308316A40026200800A3087D
:10165000031D2C2BA5010800A4017E0824020318F9
:101660003C2B83137D1883177C0824078400800893
:1016700003193C2BA40A2D2B200824020318422B0B
:101680002408A000200823020318482B2308A000E8
:10169000A401200824020318632B83137D188317E9
:1016A0007C0884000008A6008313221883172108F1
:1016B000840026088000A10A0319A20AFC0A031963
:1016C000FD0AA40A492B2308240203186E2B831356
:1016D0002218831721088400003080002408A50008
:1016E0000800A9010330F0002008BC002108BD005B
:1016F0002208BE002308BF008A1121234708A50045
:101700004808A6002508C4002608C500C601C70170
:101710008A15A61F8D2BC603C7038A1126274C08DE
:10172000AE004D08AF004E08B0004F08B100BC013C
:10173000BD01BE01BF012008C0002108C100220870
:10174000C2002308C3004A26DA088A150319C62BEB
:101750002008BC002108BD002208BE002308BF00ED
:101760002E08C0002F08C1003008C2003108C30095
:101770000130C4008A11A1274C08AA004D08AB0013
:101780004E08AC004F08AD008A15F22BA508031DCA
:10179000D62BA608031DD62B83137E1883177D082E
:1017A000290784002D308000290AA9002E08BC00DA
:1017B0002F08BD003008BE003108BF002008C0005F
:1017C0002108C1002208C2002308C3000130C40060
:1017D0008A11A1274C08AA004D08AB004E08AC00A6
:1017E0004F08AD002508BC002608BD00BE01BF01A2
:1017F0008A15A61FFD2BBE03BF030030C100B23007
:10180000C0000530C200F1214908A700A80127083F
:1018100028020318242C240829020318222C8313DD
:10182000B23084002808BC003C0884070008BD00D2
:1018300083137E1883177D08290784003D088000E4
:10184000290AA900A80A072C240829020318322C07
:1018500083137E1883177D08290784002E308000AB
:10186000290AA900A8017C0828020318A02C240832
:1018700029020318A02C2A08BC002B08BD002C0844
:10188000BE002D08BF00C001C1012030C2004130A0
:10189000C3008A11CF244E08AA004F08AB0050089D
:1018A000AC005108AD002A08BC002B08BD002C0874
:1018B000BE002D08BF0021234708A5004808A60048
:1018C0002508C4002608C500C601C7018A15A61F41
:1018D0006B2CC603C7038A1126274C08AE004D089F
:1018E000AF004E08B0004F08B1002A08BC002B081A
:1018F000BD002C08BE002D08BF002E08C0002F0818
:10190000C1003008C2003108C3000130C400A12763
:101910004C08AA004D08AB004E08AC004F08AD00C3
:101920002508303EBC0083137E1883177D082907E5
:1019300084003C088000290AA900A80A8A15332CD3
:10194000240829020318AC2C83137E1883177D0802
:1019500029078400003080002908BC0008007C08AA
:1019600083160313A1001030A200B92208008316C9
:101970000313A001A0017E082002031808008313AE
:101980007D1883177C08200784008008031908004D
:1019900083137D1883177C08200784000008A100AA
:1019A0001030A200B922A00A8A15BB2CFD08031D25
:1019B000DC2C8030FD00DE2CC030FD007C087D0773
:1019C00083160313A100A201B9220230FE008A157A
:1019D0004C2108000130FE00053083160313AC00D3
:1019E000AD012830AE0081210130FE008A155B2157
:1019F0002E08FC002F08FD00E22164308316C4008D
:101A0000C501C601C7018A1126274C08A4004D084C
:101A1000A5004E08A6004F08A7002408BC00250812
:101A2000BD002608BE002708BF000A30C000D7301E
:101A3000C1002330C2003C30C300CF244E08A400B4
:101A40004F08A5005008A6005108A7002408BC00B4
:101A50002508BD002608BE002708BF004030C00092
:101A6000DA30C1007F30C2003A30C300CF244E08C4
:101A7000A8004F08A9005008AA005108AB007C0834
:101A8000C4007D08C500C601C70126274C08A00078
:101A90004D08A1004E08A2004F08A3002008BC007A
:101AA0002108BD002208BE002308BF002808C0008E
:101AB0002908C1002A08C2002B08C300CF244E0801
:101AC000A4004F08A5005008A6005108A70024084C
:101AD000AC002508AD002608AE002708AF000800BE
:101AE000FE01053083160313AC00AD012830AE00B3
:101AF00081210130FE008A155B212E08FC002F0891
:101B0000FD00E221F4308316C4000130C500C60197
:101B1000C7018A1126274C08A4004D08A5004E08CD
:101B2000A6004F08A7002408BC002508BD00260811
:101B3000BE002708BF000A30C000D730C1002330E4
:101B4000C2003C30C300CF244E08A4004F08A500BB
:101B50005008A6005108A7002408BC002508BD00B5
:101B60002608BE002708BF004030C000DA30C100A0
:101B70007F30C2003A30C300CF244E08A8004F087F
:101B8000A9005008AA005108AB007C08C4007D08D9
:101B9000C500C601C70126274C08A0004D08A100BA
:101BA0004E08A2004F08A3002008BC002108BD0079
:101BB0002208BE002308BF002808C0002908C10071
:101BC0002A08C2002B08C300CF244E08A4004F08E7
:101BD000A5005008A6005108A7002408AC0025085D
:101BE000AD002608AE002708AF00080070252C08BD
:101BF0008312E40083162D088312E50083162E0855
:101C00008312E60083162F088312E7000A30F800DB
:101C100064088316A000831265088316A10083124E
:101C200066088316A200831267088316A300063095
:101C3000FC000030FE003430FD001430A4008A1592
:101C40007123831264088316BC008312650883160F
:101C5000BD00831266088316BE00831267088316D0
:101C6000BF007808C400C501C601C7018A11262734
:101C70004C08C0004D08C1004E08C2004F08C30008
:101C8000CF244E088312E40083164F088312E50028
:101C9000831650088312E600831651088312E7006A
:101CA00064088316A000831265088316A1008312BE
:101CB00066088316A200831267088316A300063005
:101CC000FC000030FE003430FD001430A4008A1502
:101CD00071230430F9000030FD003430FC00143072
:101CE000FE007908A0000030A2003430A1001430BA
:101CF000A30027230130FC00FD01D6240030FD00A5
:101D00003430FC001430FE00B7242030FC00AF2437
:101D10005630FC008A15AF242030FC008A15AF2411
:101D20002030FC008A15AF248A15EA242C0883127F
:101D3000DC0083162D088312DD0083162E08831223
:101D4000DE0083162F088312DF003230F8005C08B3
:101D50008316A00083125D088316A10083125E081B
:101D60008316A20083125F088316A3000630FC00CE
:101D70000030FE002030FD001430A4008A157123CD
:101D800083125C088316BC0083125D088316BD00B5
:101D900083125E088316BE0083125F088316BF009D
:101DA0007808C400C501C601C7018A1126274C085E
:101DB000C0004D08C1004E08C2004F08C300CF2428
:101DC0004E088312DC0083164F088312DD00831651
:101DD00050088312DE00831651088312DF005C086E
:101DE0008316A00083125D088316A10083125E088B
:101DF0008316A20083125F088316A3000630FC003E
:101E00000030FE002030FD001430A4008A1571233C
:101E10000430F9000030FD002030FC001430FE00DA
:101E20007908A0000030A2002030A1001430A300E7
:101E300027230030FD002030FC001430FE00B724C2
:101E40002030FC00AF244130FC008A15AF2408008C
:101E500083160313861183128611831606118312CB
:101E600006118316861083128610831606108312BD
:101E700006108316861283128612831606128312A8
:101E800006120C30FE004C213330A100A201B92211
:101E90000230FE008A154C213330A100A201B92284
:101EA0000230FE008A154C213230A100A201B92275
:101EB0000230FE008A154C212C30A100A201B9226B
:101EC0000230FE008A154C210630A100A201B92281
:101ED0000230FE008A154C210C30A100A201B9226B
:101EE0000230FE008A154C210130A100A201B92266
:101EF0000230FE008A154C210230A100A201B92255
:101F00000230FE008A154C210800073083160313A7
:101F10009F00C03081002827F625FC010530FD0018
:101F20008A15D6242A30FC00AF242A30FC008A15FA
:101F3000AF245230FC008A15AF244330FC008A15D0
:101F4000AF244C30FC008A15AF242D30FC008A15DC
:101F5000AF245230FC008A15AF244130FC008A15B2
:101F6000AF244430FC008A15AF244930FC008A15A8
:101F7000AF244F30FC008A15AF242E30FC008A15A8
:101F8000AF245230FC008A15AF245530FC008A156E
:101F9000AF242A30FC008A15AF242A30FC008A15B1
:101FA000AF24C830A1001A208A158C2FD530831297
:101FB0000313C800C430C900BB30CA00DC30CB00FA
:101FC000CC01CD01CE01CF01D001D101D201D3018D
:101FD000D401D501D601D701F201F301EB01EC01E7
:101FE000F401F501F601F701D801D901DA01DB01AD
:101FF000F001F101EF010230E000E101E201E30153
:102000008A150A12852F831203136A0E8400690E43
:0C2010008A00680E8300FF0E7F0E09009E
:02400E00723FFF
:00000001FF
